:020000040000FA
:020000000428D2
:08000800FF30A200FF30A3004D
:10001000BE01A01007309F00A410CC272214E127B6
:10002000A210E0272211DF27A211DE272212DD27EE
:10003000A212DC274030BB26A513C627A313D42762
:100040000230C400A313D4270130AD27A317D4274F
:100050000130AD27C40B22288D26201E30283228DF
:1000600041272C288B267F39A6002608A027A70029
:100070002708463C031C3F282708A800912827088A
:10008000473C031D45289A2091282708483C031D1A
:100090004C282708A80091282708493C031D52280E
:1000A000C123912827084A3C031D58282321912861
:1000B00027084C3C031D5E285321912827084D3CFE
:1000C000031D64282321912827084E3C031D6B281B
:1000D0002908A80091282708503C031D7128C32037
:1000E00091282708523C031D7728FB2291282708D6
:1000F000543C031D7D28AE2091282708563C031D43
:1001000083289F2091282708573C031D89285321C5
:1001100091282708583C031D8F28CF2391283F3072
:10012000A80001305C2727089727BD0028089726DC
:100130002C289928D226CA262708A80008002708B4
:10014000A8002030AA003130AB002E30AC00313096
:10015000AD003130AE002030AF0008002708A80005
:100160002030AA005730AB006930AC007330AD00CE
:100170007030AE003630AF003230B0003830B100F1
:100180002030B20008003D08033C031DCA2821218D
:100190000421FF283D08043C031DFC28270897265E
:1001A000A626201ED428D6284127D028BC08031D07
:1001B000DC288130BB26FA283C08013C031DE328DB
:1001C0004030BB26FA283C08023C031DEA282030B8
:1001D000BB26FA283C08033C031DF1281530BB263A
:1001E000FA283C08043C031DF8280A30BB26FA28EC
:1001F0003F30A8000329FF283F30A8000329231718
:10020000D5274030BB2E08002313D5272316D72728
:100210002513861C0C292517C7272511061E112911
:100220002515CA27861C1529C501C40AC408031D43
:100230001F29C50A4508503C031D1F2920290829EC
:100240000800AF26CA2E2708A8000A303E0203186D
:100250003F293A0EF0393B074202031D3C293C0E70
:10026000F0393D074102031D3C29380EF0393907AA
:100270004302031D3C293E29C123292952290A3062
:100280003E02031C5029380EF0393907C5003A0EDA
:10029000F0393B07C6003C0EF0393D07D625522900
:1002A0003F30A80008002708A8003E08013C031DB5
:1002B00062290230C4000430C5000830C600003096
:1002C000AC22AB2A3E08023C031D6F290330C40058
:1002D0000530C5000830C6000030AC22AB2A3E080D
:1002E000033C031D7C290230C4000430C5000830E3
:1002F000C6000030AC22AB2A3E08043C031D832913
:100300003F30A800AB2A3E08053C031D902902306F
:10031000C4000430C5001830C6001730AC22AB2A28
:100320003E08063C031D9D290330C4000530C5006E
:100330001830C6001730AC22AB2A3E08073C031920
:10034000A5293E08083C031DF8290430C4004408D0
:10035000003C031CAC29E62901304402C4000230F1
:100360004626CB01013072263108CB0004307226BC
:100370003008CB00043072262F08CB0004307226E0
:100380002E08CB0002307226CB01013072264408C1
:10039000003C0318CD29063046263208AE00360848
:1003A000B2003A08B6003308AF003708B3003B0884
:1003B000B7003408B0003808B4003C08B80035086D
:1003C000B1003908B5003D08B900A7291830462604
:1003D0003F0814273E08073C031DF1291730462625
:1003E000F3290A304626063046260430DE25AB2A9D
:1003F0003E080A3C031D292AF2250D30C800300EA4
:10040000F0393107C9002E0EF0392F072A260D309A
:10041000C800340EF0393507C900320EF039330701
:100420002A260D30C800380EF0393907C900360EBB
:10043000F03937072A260F30C8003C0EF0393D0747
:10044000C9003A0EF0393B072A2610260830DE256F
:10045000AB2A3E080B3C0319312A3E080D3C031D14
:10046000962AC8010E30C90041082A26C8016E30FC
:10047000C900A9302A26C8010E30C90042082A2620
:10048000C8016E30C900AA302A26C8010E30C90042
:100490003C0EF0393D072A26C8016E30C900A8304D
:1004A0002A26C8018430C900A6302A263E080B3C03
:1004B000031D6E2AC8010E30C90055302A26C80116
:1004C0006E30C900A7302A26C8010E30C900AA30F4
:1004D0002A26C8016E30C900A7302A26C8018230FA
:1004E000C900A6302A26C8015030C900A6302A26E5
:1004F000C8016E30C900F5302A263E080D3C031DA8
:10050000852AC801C90100302A260230CB000430F8
:10051000722606300527CB0110307226C8019430B0
:10052000C900A6302A260130DE25AB2A3E080C3C45
:10053000031DA92AF2253C0EF0393D07C4000F30F7
:10054000C8004408C90044082A2610260130DE25C8
:10055000AB2A3F30A8000800C70044084626CB015C
:10056000013072263D08CB00043072263C08CB00D7
:10057000043072263B08CB00043072263A08CB00C8
:1005800002307226CB0101307226460846263F080B
:100590001427C7080319CE2A4708462645084626C9
:1005A00001305126C80004305126AA0004305126DB
:1005B000AB0004305126AC0002305126AD000130B2
:1005C0005126C8003E08013C031DF02A3B082C02BE
:1005D000031DEE2A3A082D020319F02A3F30A80025
:1005E0003D082A02031DF82A3C082B020319FA2AA7
:1005F0003F30A80008001030C4002708A8000A30C7
:100600003E02031C052B1230C4004008C500C5087B
:10061000031D0B2BA92B3E08053C03191B2B3E0881
:10062000073C03191B2B3E08033C03191B2B3E08F8
:10063000013C031D282B0430AB234008013C031868
:10064000222BC12304305C2704304402C400A72BB2
:100650003E08043C0319342B3E08063C0319342B96
:100660003E08023C031D402B0530AB233030BA005E
:100670003030BB0004305C2704304402C400A72B98
:100680003E080A3C0319482B3E080C3C031D5B2B1B
:1006900009301F26C600460E0F398E27BC004608BB
:1006A0000F398E27BD000130DE2502305C27023075
:1006B0004402C400A72B3E080B3C0319632B3E08E1
:1006C0000D3C031DA52BC8010E30C90041082A2688
:1006D000C8016E30C900A9302A26C8010E30C900F1
:1006E00042082A26C8016E30C900AA302A26C8014D
:1006F0008030C900A6302A26C8015030C900A83071
:100700002A26C8016E30C900F5302A263E080D3C65
:10071000031D922BC801C90100302A26C801C90156
:1007200000302A2602301F26C600460E0F398E27BB
:10073000BC0046080F398E27BD000130DE2502308F
:100740005C2702304402C400A72B3F30A800C50339
:10075000072B44085C2FC600460846260130512668
:10076000C70004304B26BD0004304B26BC000430CB
:100770004B26BB0002304B26BA0001305126C70081
:1007800008000A303E020318CC2B2708A8000630C8
:1007900046260130DE25CE2B3F30A8000800270872
:1007A000A800BE010130C0003A0EF0393B07BF007F
:1007B000C301C201C1013D080C3C031D522CBC0801
:1007C0000319E62B3C08053C031DF22B0130BE004B
:1007D0006430C400DA263C08053C031DF12B0430CC
:1007E000C000512C3C08013C031DFC2B0330BE0013
:1007F0000A30C400DA26512C3C08023C031D062CAA
:100800000530BE000A30C400DA26512C3C08063CF4
:100810000319122C3C08093C0319122C3C08033C18
:10082000031D312C0A30BE000A30C400DA263C0811
:10083000033C031D1C2CC225C8018E30C900A63004
:100840002A26C8019C30C900A6302A26C501C60147
:100850000030D6253C08063C031D302C0830C00073
:10086000512C3C08043C031D3B2C0130BE00503091
:10087000C400DA26512C3C08073C0319432C3C08E1
:10088000083C031D4F2C3C08BE000A30C4003C0845
:10089000083C031D4D2C1E30C400DA26512C3F307D
:1008A000A800BC2D3D080D3C031DA92C2130C20021
:1008B000BC0803195F2C3C08083C031D652C023062
:1008C000BE006430C400DA26A82C3C08013C031D9D
:1008D0006F2C0430BE006430C400DA26A82C3C081B
:1008E000023C0319772C3C08073C031D7D2C063085
:1008F000BE006430C400DA26A82C3C08033C03196F
:10090000852C3C08093C031D9C2C0B30BE003C0888
:10091000093C031D8D2C0D30BE000A30C400C201FD
:10092000DA26C8019E30C900A6302A26C8019C30AC
:10093000C900A6302A26A82C3C08043C031DA62C7E
:100940005030C4000230BE00DA26A82C3F30A80088
:10095000BC2D3D080F3C031DFC2C2030C2003C0880
:10096000073C0319C62C3C08083C0319C62C3C085C
:10097000043C0319C62C3C08023C0319C62C3C0855
:10098000013C0319C62CBC08031DE12C0130BE003C
:10099000DA2600304626C501003037266430C40010
:1009A0003C08023C0319D82C3C08073C031DDA2CF8
:1009B0000530BE003C08013C031DE02C0330BE00A6
:1009C000FB2C3C08033C0319E92C3C08093C031DA3
:1009D000F92C0C30BE00DA26C8018E30C900A630D2
:1009E0002A26C8018C30C900A6302A260A30C40045
:1009F000FB2C3F30A800BC2D3D080E3C031DBA2D3A
:100A0000BC08031D2D2DDA26003046263F30C500D8
:100A1000FF3037260730C50006304626C50B0C2DA3
:100A20000130462607304626083046260A3005277C
:100A30000130462607304626ED2603304626C501FE
:100A4000FF303726083046260A3005270B30462669
:100A5000083046260A300527B92D3C08013C031D05
:100A6000372DDA260930462628300527B92D3C08CF
:100A7000023C03193F2D3C08073C031D4A2DDA2692
:100A800000304626C501003037261F304626053087
:100A90000527B92D3C08043C031D5E2DDA260030E5
:100AA00046263F30C500FF303726093046260A303B
:100AB00005270B3046260A300527B92D3C08083C8F
:100AC000031D722DDA26003046263F30C500FF3068
:100AD0003726093046260A3005270B3046260A30CD
:100AE0000527B92D3C08033C031D8F2DDA263C3029
:100AF000C500C6010430D6250C30C8008030C900BE
:100B000080302A26C801C90100302A26CB010430D2
:100B1000722606300527CB0110307226B92D3C080D
:100B2000093C031DB72DDA263C30C500C60105304F
:100B3000D6250C30C8000F30C9000F302A263C30B3
:100B4000C500C6010430D6250C30C8008730C90066
:100B500087302A26C801C90100302A26CB0104307B
:100B6000722606300527CB0110307226B92D3F3092
:100B7000A800BC2D3F30A800BF08031DC12D4408AC
:100B8000BF000800C8018E30C900A6302A26C8015F
:100B90008C30C900A6302A263C30C500C60106307C
:100BA000D6250C30C800C90100302A2EC7004508E0
:100BB000C3004608C2004708C100F22DC70047081D
:100BC000C800C808031DE52DF12D4127C10AC10841
:100BD000031DEF2DC20AC208031DEF2DC30AC8036F
:100BE000E12D0800C8010E30C90043082A26C801BB
:100BF0006E30C900F8302A26C8010E30C9004208FC
:100C00002A26C8016E30C900F7302A26C8010E30E6
:100C1000C90041082A26C8016E30C900F6302A2EC4
:100C2000CB0103307226A512C8272414CD273F0814
:100C300014272410CD272327CB011030722EC70094
:100C40004708CB000430722608305126C80008300F
:100C500051260800CA004808CB00043072264A0812
:100C6000CB00083072264908CB000830722EC6002F
:100C7000CB01013072264608CB00083072264508A9
:100C8000CB0006307226CB010130722EC900490814
:100C9000CB000630722EC800480851260F398E2727
:100CA0000800CA00A316D6274A08CC00CC08031DAA
:100CB0005A2E682E2414CD2741270310CB0CCB13BA
:100CC000861E632ECB172410CD274127CC03562E2A
:100CD00023274B08CD004A08083CCE00EE27CC0065
:100CE0004C080800CC00A312D6274C08CD00CD0834
:100CF000031D7B2E8A2EA5124B1C7F2EA516C827FE
:100D00002414CD270310CB0C41272410CD274127D5
:100D1000CD03772E232F1A0808009810181D922E45
:100D20004030BB2620128C1E962E20160800C400D0
:100D3000A126201E9C2E9E2E4127982E4408990005
:100D4000080020120C1EA52E20160800E8271808FF
:100D5000EB27C4002012C41CAE2E20160800A314DA
:100D6000DA272311D9272515CA27E82798019901E1
:100D7000EB2798010800C400E82724309800EB27EF
:100D80004408E8279900EB2790309800A314DA274D
:100D90002311D92FA414CC272214E127A316D62778
:100DA000D226ED2EA414CC27A01CD92E5027C83053
:100DB0000527ED2EA01CDF2E0A300527E22E562730
:100DC000C8300527A414CC272410CD27A512C82786
:100DD0002210E127A312D627ED2EA513C627A313B1
:100DE000D4272517C7272313D527A414CC270130D0
:100DF0001427A410CC2701301427A317D4270130BF
:100E000014272317D5270A30142FC5004508C6001C
:100E1000C608031D0C2F132F6430C7002327C70BF0
:100E20000E2FC603082F0800C8004808C900C908CB
:100E3000031D1B2F222F0A30CA002327CA0B1D2F88
:100E4000C903172F08002510201D272F2514CB2795
:100E500020192C2F20152D2F2011A511201D312FE9
:100E6000A515C927000000000000000000000000D8
:100E70000000000000000000000000000000000072
:100E800008002510201D452F2514CB2720194A2F97
:100E900020154B2F2011A511201D4F2FA515C92F4F
:100EA0002314DB27A315D827A01008002310DB2765
:100EB000A311D827A0140800C7004708C800C80815
:100EC000031D632F8D2F2A08A9002B08AA002C08C8
:100ED000AB002D08AC002E08AD002F08AE00300886
:100EE000AF003108B0003208B1003308B200340856
:100EF000B3003508B4003608B5003708B600380826
:100F0000B7003908B8003A08B9003B08BA003C08F5
:100F1000BB003D08BC00C8035F2F0800C90049089A
:100F2000F63E0318073E3A3EC90049080800C400CF
:100F30004408BF3E0318F93E113EC40044080800AF
:100F4000C40061304402031CAB2F44087A3C031CEC
:100F5000AB2FE030C40744080800C5004508C600B0
:100F60006430C7000A30B42FC800FF30C9004708FA
:100F7000CB004608CA00773049070318BC2FCA0BBC
:100F8000BB2FCB0BB92FC80BB72F0800CE2FCE2FFE
:100F9000CE2FCE2FCE2FCE2FD12FD12F25088600AA
:100FA0000800240885000800E22FE22FE22FE22F3C
:100FB000E22FE22FE22FE22FE52FE52FE52FE52F9D
:100FC000E52FE52F230866000800220865000800C9
:100FD000831603130800831203130800CE004E0883
:100FE000003C031CF42FFA2F0310CD0C01304E02ED
:080FF000CE00EF2F4D080800B0
:02400E00423F2F
:00000001FF
